:020000040000FA
:040000008A01032846
:0A00060083120313981383160313EB
:1000100007309C009D019B0185018601831203131B
:100020008501860101308A000030A5008316031384
:100030008600850083120313472022202F203B20B7
:1000400078201D28303084001030A40024082507B3
:100050007B208000840AA40B2628A50A0800803093
:1000600050200830A3003F30840000085C20840347
:10007000A30B35280800C03050200830A3003730CB
:10008000840000085C208403A30B4128080038305A
:10009000502001305020033050200F3050200800F5
:1000A00086006820043085006820003085006820C4
:1000B000043085006820080086006820063085002E
:1000C000682002308500682006308500682008001E
:1000D0000A30A200A100A10B6B28A20B6A2808001D
:1000E000FA30A200A100A10B7328A20B722808000D
:0800F00070207020080082005E
:100200002E34453456344F344C34553450344934FC
:100210004334203442346F346F3474346C346F346C
:1002200061346434653472342034313436344634C5
:10023000383438342E342E3434344B3420344D3466
:1002400045344D344F3452344934413420344634EB
:100250004C344134533448342E342E343334363411
:1002600038342034423459345434453453342034EF
:10027000523441344D342E342E3432343534363405
:1002800020344434453420344534453450345234D9
:100290004F344D342E342E3450345534453452348A
:1002A00054344F3453342034503441345234413474
:1002B00020344C34433444342034593420345434BE
:1002C000453443344C34413444344F342E342E348A
:1002D000523445344C3445345634413444344F342C
:1002E00052342034443445342034313432343734B9
:1002F00076342E3420343134203461346D3470340B
:100300002E342E34383420344C3445344434533471
:100310002E342E34343420344D3449344334523462
:100320004F345334573449345434433448344534C7
:1003300053342E342E34503452344F3447345234E4
:1003400041344D34413444344F34523420344434F5
:1003500045344C342034313436344634383438342F
:10036000203449344E3454344534473452344134C3
:1003700044344F342E342E34533445344E345334B5
:100380004F345234203444344534203454344534CA
:100390004D3450344534523441345434553452344D
:1003A00041342E342E345034553445345234543480
:1003B0004F342034533445345234493441344C346E
:1003C0002034523453343234333432342E342E34D5
:1003D0004634493452344D34573441345234453420
:1003E000203442344F344F3454344C344F3441343D
:1003F0004434453452342E342E342E342E342E349C
:040400002E342E3434
:00000001FF
